:0C1FF4000014000100010032000A00028D
:100D3600C10B41026B0101C00101B3004102680011
:100D4600C10AC1004102100041024500016B00C109
:100D560003C182C10841026914015600016A00C13B
:010D6600018B
:1032D000E4F5231230009002107403F0123FA13085
:1032E0000975C209900268E004F0E50DD39400402E
:1032F00010150DE50D700A1240D07F0A7E001240B5
:10330000BA786FE6600B16E6B4010620050312409A
:1033100055E510F47003E50FF4600DAF10AE0F1219
:10332000080074FFF50FF510900268E0D3940A408E
:103330000BE4F0A20B33FF1222F3B20BD2A59002E2
:103340006BE0B4051212028C7D017C007F0C121020
:103350000090026B7401F0900266E0D39413403D3C
:10336000E4F01240EA1233D7E4F569E569C3940644
:10337000502BE56925E024B5F9E790026CF0E06098
:103380001814F0E0FFE56925E024B4F8760008A6FB
:1033900007E07005AF69124083056980CE78B3E617
:1033A000700241DF16E6245BF8E614601114601A1F
:1033B000240270E9B204E4FDFF123F4880DF122AC4
:1033C000BAE4FD7F01123F4880D3123FFCE4FD7F49
:0633D00002123F4880C715
:0133D60022D4
:10300000D2D9C2A5E4F5807F01FE1240BAD2A1C296
:10301000A17F017E001240BAD2A0C2A0D2B4D2B326
:10302000D294D295D296D297C293D2B7D2B5D2B615
:10303000D2A2C2D9D2A57580FF7598507589217525
:103040008780758DFD758BFD758A04758CF7D28E22
:10305000D28CD2A943BF02123D59D2AFD2AC755324
:10306000011240EA7F507EC31240BA1240EA7F50FC
:103070007EC31240BA1240EA7F507EC31240BA1299
:1030800040EA7F507EC31240BA1240EA7F507EC3AE
:103090001240BA1240EAE4F553F524E524C3941A29
:1030A0005015E52425E02411F582E43402F583E48B
:1030B000F0A3F0052480E4E4F524E524C394025051
:1030C00009AF24122000052480F0E4FDFC7F631288
:1030D0001000E49002CAF07B017A0279677F0D123A
:1030E0003E26EF70069002677480F07B017A0279C9
:1030F0006B7F0C123E2690026BE0700E7D01FC7F10
:103100000C12100090026B7401F07D0D7C007F05A5
:103110001210007D177C007F071210007B017A02DD
:1031200079107F08123E26E4FDFF123F48E4FD7F40
:1031300002123F48E4FD7F01123F4890026BE064B9
:10314000027031FD7F04123F48E4F524E524C39466
:10315000105015E52425E02446F582E43402F58379
:10316000E4F0A3F0052480E49002CAE030E703D243
:043170000622C2066B
:013174002238
:03000B00023CB301
:103CB300C0E0C0F0C083C082C0D075D000C000C0D7
:103CC30001C002C003C004C005C006C007758A0452
:103CD300758CF7900266E004F0D20978C006E6D34B
:103CE300940440027601123AD6D007D006D005D00C
:103CF30004D003D002D001D000D0D0D082D083D062
:043D0300F0D0E032EA
:1040830078B3E6C394065007E606245BF8A6072236
:103F4800ED701FEF25E024F4F582E4341FF583E4D7
:103F580093FA740193FBEF25E024B4F8A60208A6AF
:0F3F68000322EDEF25E024B4F8760008A6052229
:103FA100900210E07008439B4075A303C2939002F6
:103FB10010E0C394014002D20A900210E0C39403BE
:053FC1004002D20022C5
:043FFC001238A622AF
:0222F3008F2436
:1022F500E4F528D20FE52414605404600261A0853A
:102305008027A2B7920CA2B5920DA2B6920EA2A2F8
:102315009210C2B7C2B5C2B6C2A27580FFC2B47F61
:102325000A7E001240BAC294858025D2947580FF3A
:10233500C295858026D295D2B4852780A20C92B706
:10234500A20D92B5A20E92B6A21092A2804D8580E2
:1023550027A2B7920CA2B5920DA2B6920EA2A29296
:1023650010C2B7C2B5C2B6C2A27580FFC2B37F059F
:102375007E001240BAC296858025D2967580FFC22E
:1023850097858026D297D2B3852780A20C92B7A2D3
:102395000D92B5A20E92B6A21092A27D01E4FCECBC
:1023A500C39408501EE5255D70028001C3500AE5FF
:1023B500265D70028001C34003ED4228ED25E0FD56
:1023C5000C80DC74672524F8E6652860237459259C
:1023D50024F80674592524F8E6C3940A401974674D
:1023E5002524F8A62874592524F8E4F6D20F800789
:1023F50074592524F8E4F674542524F8E665256017
:102405002374512524F80674512524F8E6C3940A4B
:10241500401974542524F8A62574512524F8E4F6AA
:10242500D20F800774512524F8E4F674652524F845
:10243500E66526602374572524F80674572524F885
:10244500E6C3940A401974652524F8A62674572511
:1024550024F8E4F6D20F800774572524F8E4F67DB6
:1024650001200F02A169C20FE524707CFCECC39426
:1024750008504074672524F8E65D700874A32CF8AD
:10248500E4F6802874542524F8E65D700874A32CBE
:10249500F87601801774652524F8E65D700874A345
:1024A5002CF87602800674A32CF8E4F6ED25E0FD01
:1024B5000C80BAE4900241F0A3F0FCECC394084010
:1024C50002A169900241E0FEA3E07802C333CE3356
:1024D500CED8F9F0EE900241F074A32CF8E6FFE0B7
:1024E500F0A3E04FF00C80D37C08ECC3941050406F
:1024F50074672524F8E65D700874A32CF8E4F6806B
:102505002874542524F8E65D700874A32CF8760128
:10251500801774652524F8E65D700874A32CF87699
:1025250002800674A32CF8E4F6ED25E0FD0C80BAD4
:10253500E4900243F0A3F07C08ECC394105025907E
:102545000243E0FEA3E07802C333CE33CED8F9F0E0
:10255500EE900243F074A32CF8E6FFE0F0A3E04F01
:10256500F00C80D590026BE0705AE524702C900237
:1025750041E07002A3E0601A900241E064AA700491
:10258500A3E064AA600C900241E0B45509A3E0B44D
:102595005504D203802EC203802A900243E07002C4
:1025A500A3E0601A900243E064AA7004A3E064AA61
:1025B500600C900243E0B45509A3E0B45504D2037E
:1025C5008002C20390026BE0B4030CE4FC7C10783B
:0725D500A37402F608DCFC10
:0125DC0022DC
:1033D70090026BE070183004055362FE800343626D
:1033E700013003055362FD8021436202801C3004D3
:1033F700055362FE8003436201E550D39400400702
:1034070015505362FD8003436202E4FFEFC3940843
:10341700504274A32FF8E6B4021FEF25E02431F5DC
:1034270082E43402F583E0FCA3E0D394F4EC940146
:103437004007E56113F561801874A32FF8E6B4011E
:1034470008E561C313F5618008E561C3134480F59E
:10345700610F80B8E4FFEFC39408502AEF25E024FA
:1034670021F582E43402F583E0FCA3E0D39400EC79
:1034770094024007E56313F5638008E563C31344CB
:1034870080F5630F80D0E4FFEFC39408504274AB1C
:103497002FF8E6B4021FEF25E02411F582E4340289
:1034A700F583E0FCA3E0D394F4EC94014007E564D2
:1034B70013F564801874AB2FF8E6B40108E564C30C
:1034C70013F5648008E564C3134480F5640F80B87E
:0134D70022D2
:103AD6007580FF78C0E624FE601F146031146043D1
:103AE60024037053C2B5C2B6C2A2E5536005E4F51D
:103AF600808003856180D2B722C2B7C2B6C2A2E572
:103B0600536005E4F5808003856280D2B522C2B792
:103B1600C2B5C2A2E5536005E4F5808003856380E3
:103B2600D2B622C2B7C2B5C2B6E5536005E4F58087
:083B36008003856480D2A22205
:0440EA00759FA722F5
:0B40BA00EF1FAC0670011E4C70F622D8
:1028BA0000C1814001C0804101C0804100C1814006
:1028CA0001C0804100C1814000C1814001C08041F6
:1028DA0001C0804100C1814000C1814001C08041E6
:1028EA0000C1814001C0804101C0804100C18140D6
:1028FA0001C0804100C1814000C1814001C08041C6
:10290A0000C1814001C0804101C0804100C18140B5
:10291A0000C1814001C0804101C0804100C18140A5
:10292A0001C0804100C1814000C1814001C0804195
:10293A0001C0804100C1814000C1814001C0804185
:10294A0000C1814001C0804101C0804100C1814075
:10295A0000C1814001C0804101C0804100C1814065
:10296A0001C0804100C1814000C1814001C0804155
:10297A0000C1814001C0804101C0804100C1814045
:10298A0001C0804100C1814000C1814001C0804135
:10299A0001C0804100C1814000C1814001C0804125
:1029AA0000C1814001C0804101C0804100C1814015
:1029BA0000C0C101C30302C2C60607C705C5C404D5
:1029CA00CC0C0DCD0FCFCE0E0ACACB0BC90908C845
:1029DA00D81819D91BDBDA1A1EDEDF1FDD1D1CDC35
:1029EA0014D4D515D71716D6D21213D311D1D010A5
:1029FA00F03031F133F3F23236F6F737F53534F495
:102A0A003CFCFD3DFF3F3EFEFA3A3BFB39F9F83804
:102A1A0028E8E929EB2B2AEAEE2E2FEF2DEDEC2CF4
:102A2A00E42425E527E7E62622E2E323E12120E064
:102A3A00A06061A163A3A26266A6A767A56564A454
:102A4A006CACAD6DAF6F6EAEAA6A6BAB69A9A868C4
:102A5A0078B8B979BB7B7ABABE7E7FBF7DBDBC7CB4
:102A6A00B47475B577B7B67672B2B373B17170B024
:102A7A005090915193535292965657975595945414
:102A8A009C5C5D9D5F9F9E5E5A9A9B5B9959589884
:102A9A00884849894B8B8A4A4E8E8F4F8D4D4C8C74
:102AAA0044848545874746868242438341818040E4
:090D6700016D00C111020FFFFF34
:103D5900C2D8E4786DF6786FF6FB7A00790E7F06A3
:103D69007EEF1240AEE50EF46004E50E70137B00A1
:103D79007A00790E7F06123E26EF700F750EFE80CF
:103D89000AE50EFD7C007F06121000E50E6003B403
:063D9900FF03750EFE227F
:0A40D000C2D8E4786DF6786FF6228E
:0C40A200C212D2D87F0A7E001240BA225F
:0300230002394659
:10394600C0E0C083C082C0D075D000C000C00730C0
:103956009879786DE6C394325007E6062471F8A686
:1039660099C298786DE6B40105750D328064786D5C
:10397600E66407702C7872E664036004E6B4060811
:103986009002C97408F0804A7872E6B4100B787712
:10399600E624099002C9F080399002C97432F08099
:1039A600319002C9E0FF786DE6B5070B750D00781A
:1039B6006F7606D213801B786DE6B403157872E62F
:1039C600B4190F9002C97406F08007309904C299A1
:0F39D600D212D007D000D0D0D082D083D0E03230
:10405500122E54500F7550051240A21240DA121B51
:08406500C21218001240D02223
:102E54007873E6FE08E67C002400F527EC3EF526B0
:102E64009002C9E0786D666002C3227871E6F4606E
:102E74000AE6650E6005E66002C3227872E664190C
:102E84006002E10EFB7A0079717D04123DE38E2429
:102E94008F257875E6FE08E67C002400FFEC3EFEF4
:102EA400EF65257003EE65246002C3227973E7C3DE
:102EB4007874964004E6FF80047873E6FF7973E73C
:102EC400C3787496400518E6FE80047874E6FEE53F
:102ED4000EC39F4006E50ED39E4002C322900266B5
:102EE400E0FF7E00123E9F123E687C007D14122695
:102EF4009C8D28E4F529E529C39528500B7F647E31
:102F0400001240BA052980EED3227872E664036089
:102F14000CE664066007E664106002C3227872E679
:102F24006406703CC3E5279408E526940050317884
:102F340074E6C3940250099002CAE030E022C3222E
:102F44007874E6C3940450099002CAE030E111C3D6
:102F5400227874E6B408099002CAE030E202C3227F
:102F64007873E6FE08E67C002400FFEC3EFEEF6486
:102F74000A4E703E7872E6B4030E123E687C007D01
:102F84000512269C7870A6057870E664016002C379
:102F940022123E687C007D1412269C8D28E4F529BB
:102FA400E529C39528500B7F647E001240BA052999
:102FB40080EE7B007A0079719002C9E024FEFD1254
:102FC4003DE38E248F259002C9E0246FF8E6FEE0ED
:102FD4002470F8E67C002400FFEC3EFEEFB52506E5
:072FE400EEB52402D322C365
:012FEB0022C3
:10180000E4F52CF52D7872E6B40622E4F52CE52CEF
:10181000C39408400261C17471252CF8E6F5997FE4
:10182000327E001240BA1240EA052C80E17872E65E
:1018300064036002612808E6FE08E67C002400F5E7
:1018400025EC3EF5247876E6F52A7871E6F52BF559
:1018500099C212AF2B12406D7872E6F52B3012FD53
:10186000852B99C212AF2B12406DE52A25E0F52B8E
:101870003012FD852B99C212AF2B12406DE52CC39F
:10188000952A4002610D7E00E525252CFFEE3524CA
:10189000FEEF64634E7024F52B3012FD852B99C248
:1018A00012AF2B12406D9002CAE0F52B3012FD856D
:1018B0002B99C212AF2B12406D61097E00E52525E0
:1018C0002CFFEE3524FEEF64844E7021F52B301290
:1018D000FD852B99C212AF2B12406D752B63301210
:1018E000FD852B99C212AF2B12406D61097E00E578
:1018F00025252CFFEE3524FEC3EF9464EE940050B2
:101900006BE52C2525FF7B007A007926123C00EF41
:101910007004F526F5277E00E525252CFFEE3524FD
:10192000FEC3EF945AEE94004005E4F52B8004E5E5
:1019300026F52B3012FD852B99C212AF2B12406D6C
:101940007E00E525252CFFEE3524FEC3EF945AEEEC
:1019500094004005752B018004E527F52B3012FD1E
:10196000852B99C212AF2B12406D6109AF2C7E00FE
:10197000E525252CCFEE3524CF249CCF34FFFEC3A4
:10198000EF941AEE9400505C7E00E525252CFFEEC6
:101990003524FEEF25E0FFEE33FE74492FF5827407
:1019A000013EF583E0F52B3012FD852B99C212AF75
:1019B0002B12406D7E00E525252CFFEE3524FEEF31
:1019C00025E0FFEE33FE74492FF58274013EF58366
:1019D000E0A3E0F52B3012FD852B99C212AF2B123C
:1019E000406D6109AF2C7E00E525252CCFEE352416
:1019F000CF24D4CF34FEFEC3EF94A0EE9400505019
:101A0000AF2C7E00E525252CCFEE3524CF24D4F550
:101A100029EF34FEF528AF297B007A007926753945
:101A2000011235B64006752603752778E526F52B95
:101A30003012FD852B99C212AF2B12406DE527F5B0
:101A40002B3012FD852B99C212AF2B12406D61090C
:101A5000AF2C7E00E525252CCFEE3524CF240CCFEE
:101A600034FEFEC3EF9458EE9400507DAF2C7E0000
:101A7000E525252CCFEE3524CF240CF529EF34FEB7
:101A8000F528FEAF297C007D0B1226478F2DEF75C0
:101A9000F00BA4FFC3E5299FFFE52895F0FEEF2595
:101AA000E0FFEE33FEE52D75F016A42460F582E428
:101AB0003401F583E5822FF582E5833EF583E0F579
:101AC00026A3E0F527E526F52B3012FD852B99C2DC
:101AD00012AF2B12406DE527F52B3012FD852B99A7
:101AE000C212AF2B12406D8020E4F52B3012FD8521
:101AF0002B99C212AF2B12406D752B013012FD8550
:101B00002B99C212AF2B12406D052C017D3012FDB6
:101B1000786CE6F599C2123012FD786EE6F599C23E
:101B20001230120261C180F97872E66410703AF5E1
:101B30002CE52CC39406501B7471252CF8E6F52B6C
:101B4000F599C2123012FDAF2B12406D1240EA051A
:101B50002C80DE786CE6F599C2123012FD786EE6C4
:101B6000F599C21220125A80FB7872E664197051FE
:101B700018E6F52BF599C2123012FDAF2B12406D0D
:101B80001240EA7872E6F52BF599C2123012FDAFD9
:101B90002B12406D1240EA850E2B852B99C2123014
:101BA00012FDAF2B12406D1240EA786CE6F599C237
:101BB000123012FD786EE6F599C2123012FD124015
:011BC000EA3A
:011BC1002201
:101BC200752D01C20CE4F52F7873E6FE08E67C0061
:101BD2002400F529EC3EF5287872E664066002C11D
:101BE2005408E6FE08E62400FFEC3EFEC3EF9464D0
:101BF200EE94004002A14EE6940150267876E6FD6E
:101C0200E4FF1210007875E6FD7C007F01121000DF
:101C12009002CAE04401F0E0FD7C007F63121000F4
:101C2200C1A17874E6D3940350287876E6FD7C004F
:101C32007F021210007875E6FD7C007F031210000F
:101C42009002CAE04402F0E0FD7C007F63121000C3
:101C5200C1A17874E66408702B08E6FE08E67C00F1
:101C62002400FDEC3EFC7F081210009002CAE04402
:101C720004F0E0FD7C007F631210007876E69002AB
:101C820010F0C1A17874E664057002C1A17874E60F
:101C920064077002C1A17874E6B40614E6FF787690
:101CA200E6FD7C001210007876E6F50ED20CC1A19A
:101CB2007874E6B40D14E6FF7876E6FD7C00121027
:101CC200007876E6900267F0C1A17874E6B40E124D
:101CD200E6FF7876E6FD7C001210007876E6F500E5
:101CE200C1A17874E6B40C1CE6FF7876E6FD7C00B0
:101CF2001210007876E690026BF0E06002C1A175E6
:101D02005301C1A17874E6B41012E6FF7876E6FDBD
:101D12007C001210007876E6F52DC1A17874E6B445
:101D22000A1B7870E664016002C1A17876E6FD7C48
:101D3200007F061210007876E6F50EC1A17874E6EF
:101D4200FF7876E6FD7C00121000C1A1C3E529945C
:101D52002CE52894014002A1E47873E67F00FE0896
:101D6200E67C002400FFEC3ECF249CF529EF34FFF3
:101D7200F528D3E529941AE5289400504208E6FE96
:101D820008E62400F525EC3EF524D3E52594FFE58D
:101D920024648094834002C1A17873E6FE08E6249D
:101DA20000FFEC3EFEEF25E0FFEE33FE74492FF517
:101DB2008274013EF583E524F0A3E525F0C1A1E597
:101DC20029646345286002C1A17876E6752400F58E
:101DD20025FDAC247F631210007876E69002CAF0EB
:101DE200C1A1C3E529943CE52894014002C1A17830
:101DF20073E67F00FE08E67C002400FFEC3ECF2461
:101E0200D4F529EF34FEF52808E6FE08E62400F5AD
:101E120025EC3EF524E528C313FEE529137802C319
:101E220033CE33CED8F92400F58274003EF583E533
:101E320029540125E0FFE433FEE5822FF582E58394
:101E42003EF583E524F0A3E525F085280F852910CA
:101E5200804D7872E6641070467876E6F52C7873D9
:101E6200E6FE08E67C002400F529EC3EF528E4F5C0
:101E72002AF52BC3E52B952CE52A9400502112401C
:101E8200EAE52B25E02479F8E6FD7C00E52B787461
:101E920026FF121000052BE52B7002052A80D4E5DF
:101EA2002D647F7038752E77AF2E12401DE4F52613
:101EB200E526D39410501F7B007A007927AF2612B3
:101EC2003E26EF600DE42526FDE434EEFCAF27123A
:101ED2004000052680DAC2AF759F8080FEE52DB4F2
:101EE200FF07C2AF759F8080FE300C361240EA7544
:101EF2002E77AF2E12401DE4F526E526C3940B5033
:101F02001F7B007A007927AF26123E26EF600DE490
:101F12002526FDE434EEFCAF27124000052680DAC8
:021F2200C20CEF
:011F2400229A
:0940DA00786E76FF786C76FF2207
:10406D00786CE66FFF9028BA93786E66796CF7EFEF
:05407D009029BA93F642
:01408200221B
:083DE3008B2A8A2B892C8D2DFF
:103DEB00752E00752FFF7DFFAF2D152DEF6026ABC8
:103DFB002A052CE52CAA2B7002052B14F91225DDB4
:103E0B00652FFF9028BA936D752E00F52FEF902933
:0A3E1B00BA93FD80D3E52FFEEDFF02
:013E2500227A
:030D7000011B085C
:1038A600123D9FE51B139292E51BA2E19291A2E2C3
:1038B60092907FB1123FC6123F17EF4E600412403E
:1038C600E3227F017E001240BA123EA98E198F1A9A
:1038D600123F777F017E001240BA123EA98E248FD6
:1038E60025123F777F017E001240BA123EA98E262E
:1038F6008F271240E3E51A2525FFE51935245403E1
:10390600F5288F29E51BB40815E527B52925E526F1
:10391600B528207D0FAF25AE24122CA88015E527EB
:10392600B52910E526B5280BE51B14FDAF25AE24F9
:0F393600122CA8051BE51BD3940F4003751B082B
:01394500225F
:103D9F00C2A67F017E001240BAD2A7D2A67F027EB2
:103DAF00001240BAC2A77F057E001240BAC2A67F9A
:103DBF00027E001240BAD2A7D2A67F027E00124026
:103DCF00BAC2A77F057E001240BAC2A67F027E004C
:043DDF001240BA22B2
:103F7700E4FFFE20A70B0FEF70010E64644E70F391
:103F870022D2A77F017E001240BAD2A6C2A77F0124
:093F97007E001240BAD2A7C2A6B6
:013FA00022FE
:023FC600AD0745
:103FC8007B08EB601DED3392A7D2A67F017E00121D
:103FD80040BAC2A67F017E001240BAED25E0FD1B63
:023FE80080E077
:013FEA0022B4
:103EA900E4F52AF52BFDEDC3940A502AD2A67F0129
:103EB9007E001240BAE52B25E0FFE52A33FEA2A7D2
:103EC900E433FBEEF52AEF4BF52BC2A67F017E000A
:0A3ED9001240BA0D80D0AE2AAF2BC4
:013EE30022BC
:0740E300C2A7D2A6D2A7225A
:103F1700E4F52AF52BFBFAC3EB9432EA9400501A26
:103F270020A710D2A67F017E001240BAC2A67E004B
:103F37007F00220BEB70010A80DDC2A67E007F01A5
:013F47002257
:062CA8008D2AAB07AA060D
:102CAE00E52A25E02411F582E43402F583E0FEA343
:102CBE00E0FFC3EB9FFFEA9EFE122FECD3EF94646E
:102CCE00EE648094804014E52A25E02411F582E418
:102CDE003402F583EAF0A3EBF0804CE52A25E024DC
:102CEE0011F582E43402F583E0FCA3E0C39BEC9A79
:102CFE00501074B9252AF582E43402F583E004F00D
:102D0E008025E52A25E02411F582E43402F583E0DE
:102D1E00FCA3E0D39BEC9A400E74B9252AF582E40D
:102D2E003402F583E014F074B9252AF582E43402F6
:102D3E00F583E0D36480948A501574B9252AF58200
:102D4E00E43402F583E0C3648094764002A1F5D3A7
:102D5E00EF9428EE64809480401C7C007D05122642
:102D6E009CE52A25E02411F582E43402F583EE8FEA
:102D7E00F01226D2806474B9252AF582E43402F565
:102D8E0083E0D36480948A4016E52A25E02411F569
:102D9E0082E43402F583E475F0011226D2803B748E
:102DAE00B9252AF582E43402F583E0C36480947673
:102DBE005028E52A25E02411F582E43402F583E05B
:102DCE00FEA3E04E6014E52A25E02411F582E434DA
:102DDE0002F58374FFF5F01226D274B9252AF58216
:102DEE00E43402F583E4F0E52A25E02411F582E4CB
:102DFE003402F583E0FEA3E0D39400EE9404401376
:102E0E00E52A25E02411F582E43402F5837404F0FA
:102E1E00A3E4F0E52A25E02411F582E43402F583DB
:102E2E00E0FEA3E0FFE4FCFD7B607AEAF9F8C31252
:102E3E0028875011E52A25E02411F582E43402F5A5
:052E4E0083E4F0A3F095
:012E5300225C
:0B40AE008F828E83E4931226237F0193
:0140B90022E4
:10400000AB0775F65575F6AA75F65543BF04ECF582
:0D401000F4AF058FF58BF675F7807F002269
:10401D00C2AF75F65575F6AA75F65543BF04EF2573
:0C402D00E0F5F4E4F5F575F782D2AF225F
:063D07008B4D8A4E894F2E
:103D0D001226E8FBAAF0530201EB24FFFFEA34FF71
:103D1D00FE7C007D0F122647A905EB241DFFE43A1A
:103D2D00FEE9C3EF9DFFEE9400FED3EF94FFEE94FA
:103D3D000140037F0022C3740F99FFE49400AB4D43
:0B3D4D00AA4EA94F8FF01227137F0130
:013D58002248
:063C5D008B478A488949EB
:103C63001240EAEF25E0F54A754B00854B82F58358
:103C7300E493B433037F0022054BE54B7002054AFE
:103C8300854B82854A83E493B4FF14AB47AA48A9C2
:103C930049E54A854BF012274B1240EA7F01227B0C
:0F3CA300007A00794A123D07EF70D51240EAFF10
:013CB20022EF
:0E409300EF75F0148425E025442463122623E3
:0140A10022FC
:023FEB00AC0721
:0E3FED00ED25E07B00FAAF04FC7D00124000E1
:013FFB0022A3
:0B40C500ED2401FDE43CFC1240002251
:1017ED00AE07EEB401037F0222EEB402037F0122A5
:0317FD007F002248
:083A67008F478B488A49894A08
:103A6F001240EAED25E0F54B754C00854C82F5834D
:103A7F00E493B4FF037F0022054CE54C7002054B25
:103A8F00854C82854B83E493FE740193FDEEB5471D
:103A9F0017ED6014AB48AA49A94AE54B854CF012C3
:103AAF00274B1240EA7F0122EEB4FF0AEDB4FF0666
:103ABF001240EA7F00227B007A00794B123D07EF1C
:063ACF0070BE1240EAFF88
:013AD50022CE
:0839E5008B408A4189428D43A9
:1039ED00E4F546F5471240EAE54325E0FEE42401FF
:1039FD00FFE43EF5448F45854582854483740193EC
:103A0D00FEB43314AB40AA41A942E5448545F012FA
:103A1D00274B1240EA7F0122EEB4770CE54745466D
:103A2D0070068544468545477B007A007944123DF2
:103A3D0007EF70C3E5474546700CAD43FF123FEBF2
:103A4D001240EA7F0022AB40AA41A942E5468547D4
:093A5D00F012274B1240EA7F0130
:013A6600223D
:0A367D008E408F418B428A4389443E
:103687008F828E837401937002FF221240EA854174
:1036970082854083740293F54B7F03E5412403FD44
:1036A700E43540FCEFC3940F50118D828C83E49373
:1036B700B4FF080F0DED70010C80E9EFB40F06128F
:1036C70040EA7F0022E543454460118541828540F9
:1036D70083E493AB42AA43A944122623E546454710
:1036E7006041AB45AA46A947E4F5F012274BE4F53C
:1036F7004CE54CC3954B502BAB45AA46A947122620
:10370700E875F00012274BED254CF582E43CF58374
:10371700E493FFAB45AA46A947E48FF012271305A8
:103727004C80CEE549454A600BAB48AA49A94AE512
:093737004B1226231240EA7F0127
:013740002266
:0A3B3E008B388A39893AAD07AC06CE
:103B48008D828C837401937002FF221240EA7F03F6
:103B5800ED2403FDE43CFCEFC3940F50118D828CDF
:103B680083E493B4FF080F0DED70010C80E9EFB406
:103B78000F061240EA7F0022E539453A6013AE0489
:103B8800AF058F828E83E493AB38AA39A93A1226FF
:063B9800231240EA7F0148
:013B9E002204
:083C00008F2E8B2F8A308931D1
:103C0800753501E535D3940250487B007A00793246
:103C1800853544AF2E1240937A0009AD32AF2E128B
:103C28003A67EF60297B007A007900C003C002C0C0
:103C380001852F458530468531478B488A49894A11
:103C4800D001D002D003AF34AE3312367D22053511
:043C580080B17F00B8
:013C5C002245
:083E26008F308B318A328933A1
:103E2E00753701E537D39402502D7B007A00793433
:103E3E00853744AF301240937A0009AD34AF30125B
:103E4E003A67EF600EAB31AA32A933AF36AE3512F8
:093E5E003B3E22053780CC7F00B9
:013E67002238
:0834D8008F408C418D428B43B3
:1034E0007B007A007945AD44123A67EF601BAD4628
:1034F000AC45AF42AE41123741EF700AAD46AC4524
:10350000FF1240C580037F01227B007A007945AF1E
:1035100044123C5DEF701AE54425E0F54575460020
:10352000FEAF46AD07FC7F331240001240EA7F0039
:1035300022AE45AF46AD07AC06AF40124000E543B2
:1035400075F002A4D3940CE5F0648094805013E5E8
:10355000462401FFE43545FEAD07FC7F77124000AD
:103560008011E5462401FFE43545FEAD07FC7F33BD
:10357000124000E5462402FFE43545FEAD07FCAFEE
:10358000431240007901E9D395435024AF42E5420C
:10359000E546240FFDE43545FCE9FBC3ED9BFDEC5E
:1035A0009400FC124000E541F5427541000980D6C7
:0535B0001240EA7F015A
:0135B50022F3
:083741008E478F488C498D4A28
:1037490085494C854A4D854D82854C83740193B4D6
:1037590033037F00221240EA7402254DF54DE4350A
:103769004CF54C854D82F583E493F54B054DE54DBC
:103779007002054CE4FD854D82854C83E493B4FFCA
:1037890011EDD3940C500B054DE54D7002054C0D10
:1037990080E4E54B75F002A4FFC3ED9FE5F064807A
:1037A900F87480985011E54A2401FFE43549FEADCB
:1037B90007FC7F331240007901E9D3954B501DAFC7
:1037C90048E548E9FDC3E54D9DFDE54C9400FC1233
:1037D9004000E547F5487547000980DD1240EA7F5A
:0137E90001DE
:0137EA0022BC
:061000008F308C318D32AF
:10100600E4F53EF53FD3E53294FFE5319400400523
:10101600753B028003753B017D01EDD39402505A66
:101026007B007A0079338D44AF30124093E5332547
:10103600E0F535753600853682F583E4937005AFA5
:101046003312401D853682853583E493B4FF0874D8
:101056003B2DF8E4F68020743B2DF8A605853682F4
:10106600853583E493B477028D3F85368285358353
:10107600E493B433028D3E0D80A01240EAE53C7045
:1010860027E53D7023FB7A007933754401AF3012B2
:101096004093AD337F77123FEB853344AB3BAD32A4
:1010A600AC31AF301234D822E53C6006E53D600233
:1010B6006135E53F7006E53E70026135E53F700239
:1010C60041157B007A007933F544AF301240937AAC
:1010D600007935AD33AF30123A67EF70022189AD32
:1010E60036AC35AF32AE31123741EF6002A126ADD4
:1010F60036AC35FF1240C5853344AB3BAD32AC311F
:10110600AF301234D8EF6002A126AF3F1217ED8F31
:10111600447B007A007934AF30124093AD347F7748
:10112600123FEB853444AB3BAD32AC31AF301234B9
:10113600D87B007A007935AD331239E5EF7002A11C
:10114600267B007A007937C003C0018B45754600BF
:10115600754739098B48754900894AD001D003AFD4
:1011660036AE3512367DEF7002A126853444AB3893
:10117600AD3AAC39AF371234D8AD36AC35E4FF12E0
:1011860040C522853344AB3BAD32AC31AF3012346F
:10119600D8EF6002A126AF3F1217ED8F447B007A8D
:1011A600007934AF30124093AD347F77123FEB8530
:1011B6003444AB3BAD32AC31AF301234D87B007A1D
:1011C600007935AD331239E5EF7002A1267B007A3E
:1011D600007937C003C0018B45754600754739094C
:1011E6008B48754900894AD001D003AF36AE351217
:1011F600367DEF7002A126853444AB38AD3AAC3962
:10120600AF371234D8AD36AC35E4FF1240C5227B79
:10121600007A007933853E44AF301240937A0079E4
:1012260035AD33AF30123A67EF700241BCAD36AC24
:1012360035AF32AE31123741EF6002A126AF3E1212
:1012460017ED8F447B007A007934AF30124093ADAE
:10125600347F77123FEB853444AB3BAD32AC31AFD4
:10126600301234D87B007A007935AD331239E5EF88
:101276007002A1267B007A007937C003C0018B4536
:10128600754600754739098B48754900894AD0016A
:10129600D003AF36AE3512367DEF7002A126853407
:1012A60044AB38AD3AAC39AF371234D8AD36AC357D
:1012B600E4FF1240C522AF3E1217ED8F447B007A41
:1012C600007934AF30124093AD347F77123FEB850F
:1012D6003444AB3BAD32AC31AF301234D87B007AFC
:1012E600007935AD331239E5EF7002A1267B007A1D
:1012F600007937C003C0018B45754600754739092B
:101306008B48754900894AD001D003AF36AE3512F5
:10131600367DEF7002A126853444AB38AD3AAC3940
:10132600AF371234D8AD36AC35E4FF1240C5227B58
:10133600007A007934853F44AF301240937A001921
:10134600853E44AF301240937A007935AD33AF30E5
:10135600123A67EF7002814DAD36AC35AF32AE3121
:10136600123741EF6002A126FB7A007935AD34AF22
:1013760030123A67EF6070AD36AC35AF32AE31122F
:101386003741EF6002A126853444AB3BAD32AC3128
:10139600AF301234D87B007A007935AD331239E597
:1013A600EF7002A1267B007A007937C003C0018B5B
:1013B60045754600754739098B48754900894AD0F5
:1013C60001D003AF36AE3512367DEF7002A1268509
:1013D6003444AB38AD3AAC39AF371234D8AD36AC4D
:1013E60035E4FF1240C522853444AB3BAD32AC3107
:1013F600AF301234D87B007A007935AD331239E537
:10140600EF7002A1267B007A007937C003C0018BFA
:1014160045754600754739098B48754900894AD094
:1014260001D003AF36AE3512367DEF7002A12685A8
:101436003444AB38AD3AAC39AF371234D8AD36ACEC
:1014460035E4FF1240C5227B007A007935AD34AF12
:1014560030123A67EF606EAD36AC35AF32AE311250
:101466003741EF6002A126853444AB3BAD32AC3147
:10147600AF301234D87B007A007935AD331239E5B6
:10148600EF7002A1267B007A007937C003C0018B7A
:1014960045754600754739098B48754900894AD014
:1014A60001D003AF36AE3512367DEF607385344416
:1014B600AB38AD3AAC39AF371234D8AD36AC35E4CB
:1014C600FF1240C522853444AB3BAD32AC31AF3060
:1014D6001234D87B007A007935AD331239E5EF60E6
:1014E6003F7B007A007937C003C0018B4575460003
:1014F600754739098B48754900894AD001D003AF31
:1015060036AE3512367DEF6017853444AB38AD3ACA
:10151600AC39AF371234D8AD36AC35E4FF1240C51E
:0115260022A2
:103EE4000205050506060606070707080809090A64
:103EF4000B0C0C0D0E10121315171B1E252A2F3632
:103F04003A3B37312C26231E1D1818151513111191
:033F1400100F0F7C
:0E0D73004102C600011C00C1144202C7012C3F
:102ABA00E4F524FDE51D04540FF51D90026BE0605A
:102ACA000261C8300A6C20020261C89002C6E06442
:102ADA000C7057E51C04540FF51CC202D2083014BE
:102AEA002625E02411F582E43402F5837403F0A369
:102AFA0074E8F0E51CB40702C214E49002C6F0E5DB
:102B0A0053602715538023E51C25E02411F582E440
:102B1A003402F583E4F0A3F0E51CB40702D214E40E
:102B2A009002C6F0E553600215539002C6E004F025
:102B3A0061C820020261C8E51D30E0139002C7E0B7
:102B4A00FAA3E0FBC374E89BFF74039AFE80089023
:102B5A0002C7E0FEA3E0FFC37407951D25E0241118
:102B6A00F582E43402F583EEF0A3EFF09002C6E0BA
:102B7A0064207044C202D20830141B9002C8E024B8
:102B8A0064F09002C7E03400F0E0B40320A3E0B49C
:102B9A00E81BC21480179002C8E0249CF09002C778
:102BAA00E034FFF0E07002A3E07002D214E4900275
:102BBA00C6F0E553600215539002C6E004F0E4FD46
:102BCA00EDC39408504474A32DF8E6B40221ED2510
:102BDA00E02431F582E43402F583E0FAA3E0D394E9
:102BEA00F4EA94014009E526134480F52680187416
:102BFA00A32DF8E6B4010AE526C3134480F526801E
:102C0A0006E526C313F5260D80B67D08EDC394109C
:102C1A00504474A32DF8E6B40221ED25E02401F511
:102C2A0082E43402F583E0FAA3E0D394F4EA94014F
:102C3A004009E525134480F525801874A32DF8E68C
:102C4A00B4010AE525C3134480F5258006E525C3AA
:102C5A0013F5250D80B6AD80A2B7920CA2B5920DE0
:102C6A00A2B6920EA2A2920FC2B7C2B5C2B6C2A2B1
:102C7A007580FF300A15E51D30E009852580D2A14F
:102C8A00C2A18007852680D2A0C2A08D80A20C9204
:0D2C9A00B7A20D92B5A20E92B6A20F92A2A3
:012CA700220A
:041F25008E088F098A
:101F2900E4F50A903EE493750B00F50CD3E50C95A6
:101F390009E50B95084006E4FAFBFFFE22050AAF06
:101F49000AEF3395E0FE74E42FF582743E3EF58383
:101F5900E493250CF50CE4350BF50BD3E50C950949
:101F6900E50B95084078E50C9509FFE50B9508FE0A
:101F7900AD0AED3395E0FC74E42DF582743E3CF531
:101F890083E493C39FFBE49EFA7C007D0AAF03FEC2
:101F9900122635AA06AB07AF0AEF3395E0FE74E4C3
:101FA9002FF582743E3EF583E493FDAF03AE021232
:101FB900269CAA06AB077C007D051226357D0A12F0
:101FC900269CAA06AB07AF0AEF3395E0FE7C007D9D
:101FD90005122635EF2BFBEE3AFAAF03FE22E50A8E
:0A1FE9006002E146FA7BFF7FFFFE75
:011FF30022CB
:100D810061400020000000000000000000000000A1
:100D91000000000000000000000000000000000052
:100DA1000000000000000000000000000000000042
:100DB1000000000000000000000000000000000032
:100DC1000000000000000000000000000000000022
:100DD1000000000000000000000000000000000012
:100DE1000000000000000000000000000000000002
:100DF10000000000000000000000000000000000F2
:100E010000000000000000000000000000000000E1
:100E110000000000000000000000000000000000D1
:100E210000000000000000000000000000000000C1
:100E310000000000000000000000000000000000B1
:100E410000000000000000000000000000000000A1
:100E51000000000000000000000000000000000091
:100E61000000000000000000000000000000000081
:100E71000000000000000000000000000000000071
:100E81000000000000000000000000000000000061
:100E91000000000000000000000000000000000051
:100EA1000000000000000000000000000000000041
:100EB1000000000000000000000000000000000031
:100EC1000000000060B001600000000000000000B0
:100ED1000000000000000000000000000000000011
:100EE1000000000000000000000000000000000001
:100EF10000000000000000000000000000000000F1
:100F010000000000000000000000000000000000E0
:100F110000000000000000000000000000000000D0
:100F210000000000000000000000000000000000C0
:100F310000000000000000000000000000000000B0
:100F410000000000000000000000000000000000A0
:100F51000000000000000000000000000000000090
:100F61000000000000000000000000000000000080
:100F710000000000000000006020000004010401E6
:100F81000401040104010401040104010401040138
:0C0F910004010401040104010401040136
:10028C00E4F5247D02FC7F02123800E4F524E52419
:10029C00C394084002E1DB1240EA75F028E524A47F
:1002AC002420F582E5F03400F583E0FEA3E04E70E7
:1002BC004A75F028E524A42422F582E5F03400F5F3
:1002CC0083E0FEA3E04E703375F028E524A42424CB
:1002DC00F582E5F03400F583E0FEA3E04E701C756A
:1002EC00F028E524A42426F582E5F03400F583E01B
:1002FC00FEA3E04E7005752501E1D775F028E524C5
:10030C00A42420F582E5F03400F583E0FEA3E04E52
:10031C00703B75F028E524A42422F582E5F0340026
:10032C00F583E0FEA3E0FFE52475F016A42460F548
:10033C0082E43401F583EEF0A3EFF0752602752705
:10034C0001E4753364F532F531F5308166E52475D9
:10035C00F016A42460F582E43401F583E4F0A3F0F4
:10036C00F526752701753364F532F531F53075F0E6
:10037C0028E524A42420F582E5F03400F583E0FE82
:10038C00A3E0FFE4FCFDAB33AA32A931A830D312B1
:10039C00289D40028163E47FE87E03FDFCA83012B7
:1003AC00289D4002816375F028E524A42420F58261
:1003BC00E5F03400F583E0FEA3E0FFC3E49FFFE427
:1003CC009EFE122FEC8E288F2975F028E524A4248C
:1003DC0022F582E5F03400F583E0FEA3E0FFC3E4F0
:1003EC009FFFE49EFE122FEC8E2A8F2BE4FCFDABBC
:1003FC0033AA32A931A83012276AC004C005C0063E
:10040C00C007AE28AF29E4FCFDF8F9AA06AB07D06B
:10041C0007D006D005D0041227F58F2F8E2E8D2DE8
:10042C008C2CE52475F016A42460F582E43401F5D7
:10043C008375F002E5271228AEEEF0A3EFF0052746
:10044C00E5332464F533E43532F532E43531F531F6
:10045C00E43530F530617A75260275F028E524A470
:10046C002420F582E5F03400F58375F002E52612C0
:10047C0028AEE0FEA3E0FFE4FCFDAB33AA32A931C9
:10048C00A830D312289D4002C141E47FE87E03FDD1
:10049C00FCA83012289D4002C141E526C3941440AB
:1004AC0002C14175F028E524A4241CF582E5F03442
:1004BC0000F58375F002E5261228AEE0FEA3E0FFFE
:1004CC0075F028E524A42420F582E5F03400F583AA
:1004DC0075F002E5261228AEE0FCA3E0C39FFFEC0A
:1004EC009EFE122FEC8E288F2975F028E524A4246B
:1004FC001EF582E5F03400F58375F002E52612282E
:10050C00AEE0FEA3E0FF75F028E524A42422F582DA
:10051C00E5F03400F58375F002E5261228AEE0FC18
:10052C00A3E0C39FFFEC9EFE122FEC8E2A8F2B753F
:10053C00F028E524A4241CF582E5F03400F583753D
:10054C00F002E5261228AEE0FEA3E0FFE4FCFDC3BA
:10055C00E5339FFBE5329EFAE5319400F9E53094E2
:10056C0000F8AE2AAF2BE412276AC004C005C006FF
:10057C00C007AE28AF29E4FCFDF8F9AA06AB07D0FA
:10058C0007D006D005D0041227F5A804A905AA06A1
:10059C00AB0775F028E524A4241EF582E5F03400A1
:1005AC00F58375F002E5261228AEE0FEA3E0FFE429
:1005BC00FCFDEB2FF52FEA3EF52EED39F52DEC3841
:1005CC00F52CE52475F016A42460F582E43401F5CD
:1005DC008375F002E5271228AEE52EF0A3E52FF087
:1005EC000527E5332464F533E43532F532E435314F
:1005FC00F531E43530F53075F028E524A42420F5E8
:10060C0082E5F03400F58375F002E5261228AEE0A1
:10061C00FEA3E0FFE4FCFDAB33AA32A931A830D332
:10062C0012289D50028166E52694144002816605CD
:10063C0026052680C2E526C394145002E1D7E47F38
:10064C00E87E03FDFCAB33AA32A931A830D31228C3
:10065C009D4002E1D7E52475F016A42474F582E4DC
:10066C003401F5837403F0A374E8F075F028E524E5
:10067C00A42420F582E5F03400F58375F002E5261C
:10068C001228AEE0FEA3E04E70061526152680DB80
:10069C00E47FE87E03FDFCAB33AA32A931A830D34A
:1006AC0012289D4002E1D775F028E524A42420F5FA
:1006BC0082E5F03400F58375F002E5261228AEE0F1
:1006CC00FEA3E0FFC374E89FFF74039EFE122FECA1
:1006DC008E288F2975F028E524A42422F582E5F0D4
:1006EC003400F58375F002E5261228AEE0FEA3E097
:1006FC00FFC374E89FFF74039EFE122FEC8E2A8FAB
:10070C002B75F028E524A42420F582E5F03400F5BF
:10071C008375F002E5261228AEE0FEA3E0FFE4FCB0
:10072C00FDC3E5339FFBE5329EFAE5319400F9E514
:10073C00309400F8AE2AAF2BE412276AC004C0052F
:10074C00C006C007AE28AF29E4FCFDF8F9AA06AB39
:10075C0007D007D006D005D0041227F5A804A905A8
:10076C00AA06AB0775F028E524A42422F582E5F04F
:10077C003400F58375F002E5261228AEE0FEA3E006
:10078C00FFE4FCFDEB2FF52FEA3EF52EED39F52DB0
:10079C00EC38F52CE52475F016A42460F582E434CD
:1007AC0001F58375F002E5271228AEE52EF0A3E5DE
:1007BC002FF00527E5332464F533E43532F532E4C4
:0F07CC003531F531E43530F530C19C0524419AC3
:0107DB0022FB
:063800008C348D35AB078E
:103806007A05EA75F064A4FFD3E5359FE53495F0B3
:1038160040030A80EDEA75F064A4FFC3E5359FE531
:103826003495F050031A80EDEB75F016A42460F57C
:1038360082E43401F58375F002EA1228AEE0FEA3B5
:10384600E0FFEB75F016A42462F582E43401F583FB
:1038560075F002EA1228AEE0FCA3E0C39FF537EC50
:103866009EF536EA75F064A4FFC3E5359FFFE5349F
:1038760095F0FEAC36AD371226357C007D641226F7
:1038860047EB75F016A42460F582E43401F58375E0
:0F389600F002EA1228AEE0FCA3E02FFFEC3EFEAA
:0138A5002200
:10080000EEC313EF13F52475F014A4F526E52425A3
:10081000E025E02400F582E43400F583E0FEA3E067
:10082000C39401EE94044002A135E52425E025E0BF
:100830002402F582E43400F583E0FEA3E0C39401D2
:10084000EE94044002A135E5262412FF7B007A00D5
:1008500079277539011235B64006752704752801C8
:10086000E52864017004E52764046002614F752582
:1008700010E5262525FF7B007A00792775390112BE
:1008800035B64006752704752801E525D394004048
:100890002CE5289401E527940440221240EA15250E
:1008A0001525E5262525FF7B007A00792775390176
:1008B0001235B640D575270475280180CDE5256031
:1008C000024102E52864017004E5276404703AE5FA
:1008D0002425E025E02400F582E43400F583E0FCE3
:1008E000A3E0FD7B01AF26123B9FE52425E025E038
:1008F0002402F582E43400F583E0FCA3E0FDE52664
:1009000004FF7B01123B9FA109E52425E025E0249B
:1009100000F582E43400F583E0FEA3E0C39528EE01
:1009200095275066E5262402FF7B01AD28AC2712EF
:100930003B9FE52604FF7B007A0079277539011279
:1009400035B6E5262403FF7B01AD28AC27123B9F7B
:10095000E52425E025E02400F582E43400F583E079
:10096000FCA3E0FD7B01AF26123B9FE52425E0259B
:10097000E02402F582E43400F583E0FCA3E0FDE529
:100980002604FF7B01123B9FA109E52425E025E019
:100990002400F582E43400F583E0FEA3E0D395283B
:1009A000EE9527403EE52425E025E02400F582E48D
:1009B0003400F583E0FCA3E0FDE5262402FF7B0183
:1009C000123B9FE52425E025E02402F582E4340073
:1009D000F583E0FCA3E0FDE5262403FF7B01123B49
:1009E0009FA109E52425E025E02402F582E43400F6
:1009F000F583E0FCA3E0FDE52604FF7B01123B9FAD
:100A0000A109E526FD7C00AB24AF2512173F40026B
:100A1000A109E52425E025E02400F582E43400F571
:100A200083E0F52BA3E0F52CE5262525FF7B007A56
:100A30000079277539011235B6D3E528952CE527BD
:100A4000952B4053E525D39400404C1240EAE5260F
:100A500025252402FF7B01AD28AC27123B9FE5260C
:100A6000252504FF7B007A0079277539011235B6F8
:100A7000E52625252403FF7B01AD28AC27123B9FEB
:100A800015251525E5262525FF7B007A0079277594
:100A900039011235B680A2E5257071D3E528952C71
:100AA000E527952B4066E5262402FF7B01AD28ACA7
:100AB00027123B9FE52604FF7B007A0079277539D2
:100AC000011235B6E5262403FF7B01AD28AC2712C1
:100AD0003B9FE52425E025E02400F582E43400F581
:100AE00083E0FCA3E0FD7B01AF26123B9FE52425BC
:100AF000E025E02402F582E43400F583E0FCA3E085
:100B0000FDE52604FF7B01123B9FA1090525052574
:100B1000E52425E025E02400F582E43400F583E0B7
:100B2000FCA3E0FDE5262525FF7B01123B9FE52484
:100B300025E025E02402F582E43400F583E0FCA3FF
:100B4000E0FDE526252504FF7B01123B9FA109124C
:100B500040EAE4F525E5262525FF7B007A00792784
:100B60007539011235B6E52425E025E02400F5822B
:100B7000E43400F583E0FEA3E0D39528EE9527400A
:100B80001DE5259414501705250525E5262525FF87
:100B90007B007A0079277539011235B680C8E525C2
:100BA00064147041E52425E025E02400F582E43456
:100BB00000F583E0FCA3E0FDE526252524FEFF7B70
:100BC00001123B9FE52425E025E02402F582E43470
:100BD00000F583E0FCA3E0FDE526252514FF7B015D
:100BE000123B9FA109E525703FE52425E025E0247F
:100BF00000F582E43400F583E0FCA3E0FDE5262562
:100C000025FF7B01123B9FE52425E025E02402F52A
:100C100082E43400F583E0FCA3E0FDE5262525040D
:100C2000FF7B01123B9FA109E5262525FF7B007A6A
:100C30000079277539011235B6E526252524FEFFF2
:100C40007B007A0079297539011235B6E52425E053
:100C500025E02400F582E43400F583E0FEA3E0FF04
:100C6000C3E5289FFFE5279EFEE52425E025E02437
:100C700000F582E43400F583E0FCA3E0C3952AFD8F
:100C8000EC9529FCC3EF9DEE9C503FE52425E02523
:100C9000E02400F582E43400F583E0FCA3E0FDE508
:100CA000262525FF7B01123B9FE52425E025E02436
:100CB00002F582E43400F583E0FCA3E0FDE526259F
:100CC0002504FF7B01123B9F803FE52425E025E0C2
:100CD0002400F582E43400F583E0FCA3E0FDE52682
:100CE000252524FEFF7B01123B9FE52425E025E01E
:100CF0002402F582E43400F583E0FCA3E0FDE52660
:100D0000252514FF7B01123B9FE52425E025E024E7
:100D100000F582E43400F5837404F0A37401F0E577
:100D20002425E025E02402F582E43400F5837404F0
:050D3000F0A37401F0C6
:010D3500229B
:06173F008C2D8D2E8B2F76
:10174500EF24FEF530E52F25E025E02400F582E4C1
:101755003400F583E0F531A3E0F532E530252EFFC1
:101765007B007A0079337539011235B6E532653477
:101775007004E5316533601EE530D39400401715DC
:10178500301530E530252EFF7B007A007933753929
:10179500011235B680D6E530702DE532653470041A
:1017A500E53165336002D322E52F25E025E02402EB
:1017B500F582E43400F583E0FCA3E0FDE52E04FFAB
:1017C5007B01123B9FC322E52F25E025E02402F58E
:1017D50082E43400F583E0FCA3E0FDE530252E042A
:0717E500FF7B01123B9FC3D3
:0117EC0022DA
:100F9D004402B3020002004802AB0068006900661B
:090FAD0000674402A300020002E7
:1007DC00AB07C2AF75F65575F6AA75F65543BF044F
:1007EC00ECF5F4AF058FF58BF675F780D2AF7F0083
:0107FC0022DA
:10403900C2AF75F65575F6AA75F65543BF04EF2557
:0C404900E0F5F4E4F5F575F782D2AF2243
:1037EB001226E8F58285F083E4932402FFE4338FFD
:0537FB00F0122713226B
:020FB700A90788
:100FB900E925E024A3F582E43402F583E0A3E0F512
:100FC9003BE925E02411F8E6FE08E6FFE53B2402AB
:100FD900FDE433FCE925E024A7F582E43402F58336
:100FE900E0FAA3E0C39DFDEA9CFCD3EF9DEE9C4093
:040FF90002D322C33A
:010FFD0022D1
:022000008F252A
:10200200EF25E024B3F582E43402F583E0F528A35A
:10201200E0F529EF25E025E024ABF582E43402F572
:1020220083E0A3E0F526EF25E025E024ADF582E488
:102032003402F583E0A3E0F527E52625E0F52A75CD
:102042002B00E52725E0752CFFF52D752E00852B3D
:1020520082852A83E4936455600221DAAB2CAA2D8F
:10206200A92E1225DD6455600221DAE52B2401FF39
:10207200E4352AFEE52525E02411F8A60608A60780
:10208200E52525E02411F8E6FE08E6F5828E83E4D4
:1020920093F46036AB2CAA2DA92EC0038A838982C1
:1020A200E52525E02411F8E6FE08E6AA06F9C3D0E4
:1020B200E0E99582EA95835011E52575F002A424A2
:1020C20011F9E4FAFB1237EB80B6E52525E024117D
:1020D200F8E6FE08E6C3952BF530EE952AF52FE5D6
:1020E2002E2401F9E4352DFEAF01E52525E024116A
:1020F200F8A60608A607E52525E02411F8E6FE085D
:10210200E6F5828E83E493F4603CAB2CE52E252920
:10211200F9E52D3528FAC0038A838982E52525E071
:102122002411F8E6FE08E6AA06F9C3D0E0E9958292
:10213200EA95835011E52575F002A42411F9E4FA19
:10214200FB1237EB80B0E52525E02411F8E6FE0806
:10215200E6C3952EFFEE952DFED3EF9530EE952F2B
:10216200503DE52E2401FFE4352DFEE52525E02432
:102172009FF582E43402F583EEF0A3EFF074B72505
:1021820025F582E43402F583E526F0AE2AAF2BADC5
:1021920007AC06E4FF1207DCEF70024184C322E5BC
:1021A2002B2401FFE4352AFEE52525E0249FF58254
:1021B200E43402F583EEF0A3EFF074B72525F5823F
:1021C200E43402F583E527F0AC2DAD2EE4FF1207CF
:1021D200DCEF70024184C322852B82852A83E4933B
:1021E200B4552BE52B2401FFE4352AFEE52525E035
:1021F200249FF582E43402F583EEF0A3EFF074B786
:102202002525F582E43402F583E527F08074AB2CB2
:10221200AA2DA92E1225DDB4552DAE02AF01EF2451
:1022220001FFE43EFEE52525E0249FF582E4340229
:10223200F583EEF0A3EFF074B72525F582E43402BE
:10224200F583E526F0803BE52B2401FFE4352AFEE9
:10225200E52525E0249FF582E43402F583EEF0A320
:10226200EFF074B72525F582E43402F583E527F013
:10227200AE2AAF2BAD07AC067F551207DCEF60022A
:10228200C322E52525E0249FF582E43402F583E0AC
:10229200FEA3E0FFE52525E02411F8A60608A6071F
:1022A200E52525E0249FF582E43402F583E0FEA3D0
:1022B200E02529FFE5283EFEE52525E024A7F58255
:1022C200E43402F583EEF0A3EFF0E52525E02411D6
:1022D200F8E6FE08E6F5828E83E493F46011E525C4
:1022E20075F002A42411F9E4FAFB1237EB80DBD378
:0122F20022C9
:021527008F3BF8
:10152900EF25E0249FF582E43402F583E0FEA3E091
:101539008E3CF53D74B72FF582E43402F583E0253E
:10154900E0F53E753F00E53B25E024B3F582E43440
:1015590002F583E0FFA3E09002C4CFF0A3EFF0E42B
:101569009002C1F09002C4E0C313FF9002C1E0C32E
:101579009F50201240EA74B7253BF582E43402F506
:1015890083E0FF9002C1E0FEEF2EFF124039E00434
:10159900F080D1053FE53F7002053E853D82853CDF
:1015A90083E493F47002C16A1240EA853D82853C66
:1015B900837401937002C15F740193F47002C15F77
:1015C900053DE53DAE3C7002053C14F5828E83E491
:1015D900939002C2F0E0FFAC3EAD3F1207DCEF6032
:1015E900037F0122053FE53F7002053E053DE53DCC
:1015F900AE3C7002053C14F5828E83E493FFAC3E49
:10160900AD3F1207DCEF60037F0122053FE53F7024
:1016190002053EE49002C1F09002C2E0FF9002C1CF
:10162900E0C39F4002A1A4053DE53DAE3C70020523
:101639003C14F5828E83E493FFAC3EAD3F1207DC88
:10164900EF60037F0122053FE53F7002053E9002EE
:10165900C1E004F080C27B007A00793C1237EBA12B
:10166900A4E53B25E02411F8A63E08A63FE53B2565
:10167900E0249FF582E43402F583E0C3139002C3AA
:10168900F074B7253BF582E43402F583E025E0FEEA
:10169900E53B25E0249FF582E43402F583EEF0A3CF
:1016A900E4F09002C3E0FF74B7253BF582E434020D
:1016B900F583EFF0E53B25E0249FF582E43402F55C
:1016C90083E0FEA3E0FF9002C4E0FCA3E0FDEF2D60
:1016D900FFEE3CFEE53B25E024A7F582E43402F564
:1016E90083EEF0A3EFF0E53B25E0249FF582E43497
:1016F90002F583E0FCA3E0FD7F551207DCEF6003F0
:101709007F012274B7253BF582E43402F583E07D3D
:101719000025E0FCE4FF1207DCEF60037F0122E50E
:101729003B25E0249FF582E43402F583E475F0015A
:051739001226D27F0022
:01173E002288
:083175008F3B8B3C8A3D893E33
:10317D00E4F544F545E53F25E024A3F582E434026A
:10318D00F583E0A3E0F546E53F25E0249FF582E4D5
:10319D003402F583E0FEA3E08E40F541053BE53FAB
:1031AD0025E02411F8E6FE08E6FFE5462401FDE4DE
:1031BD0033FCE53F25E024A7F582E43402F583E0F6
:1031CD00FAA3E0C39DFDEA9CFCD3EF9DEE9C40016C
:1031DD0022854182854083740193653B6010E493A1
:1031ED00F4600B7B007A0079401237EB80E3854168
:1031FD0082854083740193B53B0BE5412401F54570
:10320D00E43540F544E53F25E02411F8E6FE08E6F7
:10321D00FFFDAC06AF461207DC8F42E5426002C3EC
:10322D0022E53F25E02411F808740226F618E4364D
:10323D00F6E4F543E543C395465033E53F25E024D9
:10324D0011F8E6FE08E62543FFE43EFEAD07FCABB4
:10325D003CAA3DA93E8543827583001225F6FF12D7
:10326D0007DC8F42E5426002C322054380C6E53F7D
:10327D0025E02411F808E54626F618E436F6E53F74
:10328D0025E02411F8E6FE08E6FFE5462401FDE4FD
:10329D0033FCC3EF9DFFEE9CFEAD07FCAF3B120769
:1032AD00DC8F42E5426002C322E54545446012AE23
:1032BD0044AF45AD07AC06E4FF1207DCEF6002C377
:0232CD0022D30A
:0132CF0022DC
:0835B6008F358B368A37893806
:1035BE00E53925E0249FF582E43402F583E0FEA38D
:1035CE00E08E3AF53BE4F53CF53D0535853B8285CD
:1035DE003A83E493F46053E53925E024A7F582E4B9
:1035EE003402F583E0FCA3E0D3953BEC953A403AE8
:1035FE00853B82853A8374019365357022E53D459E
:10360E003C6016E53D2401FFE4353CFEAD07FCE4CD
:10361E00FF1207DCEF6002C322853A3C853B3D7BFF
:10362E00007A00793A1237EB80A2E53D453C603DC9
:10363E00853D82853C83740293FFAB36AA37A93849
:10364E00E48FF012274BAB36AA37A9381226E8754D
:10365E00F00012274B853D82853C83740393FFABAC
:0E366E0036AA37A938E48FF0122713D322C3EF
:01367C00222B
:043B9F008F358B369D
:103BA300E4F537EDF539ECF5381240EAAF36120F8C
:103BB300B75025E537C3940A500CAF36121527EFDB
:103BC3006004053780ED7F057E001240BAE537C3F8
:103BD300940A400122E4F537E537C3940A50147B75
:103BE300007A00793885363FAF35123175400405C8
:0C3BF3003780E5E537C3940A400122D377
:013BFF0022A3
:03000000020200F9
:0C020000787FE4F6D8FD7581C00202474B
:1025DD00BB010689828A83E0225002E722BBFE02FC
:0925ED00E32289828A83E493222F
:1025F600BB010CE58229F582E5833AF583E022509A
:1026060006E92582F8E622BBFE06E92582F8E222E3
:0D261600E58229F582E5833AF583E49322FD
:10262300BB010689828A83F0225002F722BBFE0196
:02263300F32290
:10263500EF8DF0A4A8F0CF8CF0A428CE8DF0A42EB9
:02264500FE2273
:10264700BC000BBE0029EF8DF084FFADF022E4CC77
:10265700F875F008EF2FFFEE33FEEC33FCEE9DEC40
:10266700984005FCEE9DFE0FD5F0E9E4CEFD22ED86
:10267700F8F5F0EE8420D21CFEADF075F008EF2FD0
:10268700FFED33FD4007985006D5F0F222C398FDC1
:052697000FD5F0EA225E
:10269C00C2D5EC30E709B2D5E4C39DFDE49CFCEE59
:1026AC0030E715B2D5E4C39FFFE49EFE122647C364
:1026BC00E49DFDE49CFC800312264730D507C3E45F
:0626CC009FFFE49EFE22C8
:1026D200C5F0F8A3E028F0C5F0F8E5821582700293
:0626E2001583E038F02230
:1026E800BB010A89828A83E0F5F0A3E022500687BD
:1026F800F009E71922BBFE07E3F5F009E31922897F
:0B270800828A83E493F5F074019322B1
:10271300BB010789828A830226D2500B09C5F027A1
:10272300F7C5F01937F722BBFE0D09F8E325F0F3DF
:10273300C5F019E338F322F889828A83740193255B
:08274300F0C5F0F8E493382220
:10274B00BB010A89828A83F0E5F0A3F0225006F7D9
:0F275B0009A7F01922BBFE06F3E5F009F31922D6
:10276A00E88FF0A4CC8BF0A42CFCE98EF0A42CFC0E
:10277A008AF0EDA42CFCEA8EF0A4CDA8F08BF0A48C
:10278A002DCC3825F0FDE98FF0A42CCD35F0FCEBEB
:10279A008EF0A4FEA9F0EB8FF0A4CFC5F02ECD39B0
:0F27AA00FEE43CFCEAA42DCE35F0FDE43CFC221D
:1027B90075F008758200EF2FFFEE33FECD33CDCCD7
:1027C90033CCC58233C5829BED9AEC99E58298405A
:1027D9000CF582EE9BFEED9AFDEC99FC0FD5F0D637
:1027E900E4CEFBE4CDFAE4CCF9A88222B800C1B961
:1027F9000059BA002DEC8BF084CFCECDFCE5F0CB9F
:10280900F97818EF2FFFEE33FEED33FDEC33FCEBD7
:1028190033FB10D703994004EB99FB0FD8E5E4F992
:10282900FA227818EF2FFFEE33FEED33FDEC33FC7F
:10283900C933C910D7059BE99A4007EC9BFCE99A73
:10284900F90FD8E0E4C9FAE4CCFB2275F010EF2FB8
:10285900FFEE33FEED33FDCC33CCC833C810D707B8
:102869009BEC9AE899400AED9BFDEC9AFCE899F8F3
:0E2879000FD5F0DAE4CDFBE4CCFAE4C8F92286
:10288700EB9FF5F0EA9E42F0E99D42F0EC6480C8C8
:0628970064809845F02268
:10289D00EB9FF5F0EA9E42F0E99D42F0E89C45F091
:0128AD002208
:0C28AE00A42582F582E5F03583F5832235
:103E6800AC15AD16AE17AF18780FEFA2E2EC20E64E
:103E780001B35D5E5FF47004FCFDFEFFEF13FFEE1F
:103E880013FEED13FDEC13FCD8E08C158D168E1780
:103E98008F18EE547FFE228E158F16E4F517F5184D
:013EA80022F7
:102FEC00C3EE6480948040028007C3E49FFFE49E9C
:022FFC00FE22B3
:10020C000232D0E493A3F8E493A34003F68001F206
:10021C0008DFF48029E493A3F85407240CC8C333F3
:10022C00C4540F4420C8834004F456800146F6DFC2
:10023C00E4800B0102040810204080900D36E47E0F
:10024C00019360BCA3FF543F30E509541FFEE493B7
:10025C00A360010ECF54C025E060A840B8E493A37E
:10026C00FAE493A3F8E493A3C8C582C8CAC583CAA9
:10027C00F0A3C8C582C8CAC583CADFE9DEE780BE61
:010FB600003A
:00000001FF
